:1000000012C02AC029C028C027C026C025C024C0CD
:1000100023C022C021C020C01FC01EC01DC01CC0E4
:100020001BC01AC019C011241FBECFEDCDBF10E0F8
:10003000A0E6B0E0ECEEF0E002C005900D92A03733
:10004000B107D9F710E0A0E7B0E001C01D92A237D8
:10005000B107E1F73DD048C0D3CFE0917000609187
:10006000710044E1F0E0E05AFF4F8FEF90E0861B13
:10007000910918C0308138BB36E03A95F1F700C0DD
:100080002F5F2617B8F350E006C018BA26E02A956D
:10009000F1F700C05F5F252F30E028173907ACF378
:1000A000415011F020E0EDCF08951F9310E0109320
:1000B0007100D3DF1F5F1A3FD1F71F9108951F937F
:1000C0001AEF10937100C9DF1150D9F71F910895ED
:1000D0001F938FE787BB10E010937000E6DFEFDF20
:0C00E0001F5F1031C0F7F8CFF894FFCF7D
:1000EC007B036E4F175D7D0B7F5F3F7578677C3CA4
:00000001FF
